:060000000C94CE000C94EC
:1000060000000C9400000C9400000C9400000C946A
:1000160000000C9400000C94FE000C9400000C945C
:1000260000000C9400000C9400000C9400000C944A
:1000360000000C9400000C9400000C9400000C943A
:1000460000000C9400000C9400000C9400000000CA
:10005600000000000000000000000000000000009A
:10006600000000000000000000000000000000008A
:10007600000000000000000000000000000000007A
:10008600000000000000000000000000000000006A
:10009600000000000000000000000000000000005A
:1000A600000000000000000000000000000000004A
:1000B600000000000000000000000000000000003A
:1000C600000000000000000000000000000000002A
:1000D600000000000000000000000000000000001A
:1000E600000000000000000000000000000000000A
:1000F60000000000000000000000000000000000FA
:1001060000000000000000000000000000000000E9
:1001160000000000000000000000000000000000D9
:1001260000000000000000000000000000000000C9
:10013600000000000000000000000000000000FFBA
:100146004108413C410000804114411841000080B3
:10015600412241186300008041414118550000FFCB
:100166007F7F7F18490000FF7F7F7F1841000001D5
:10017600414141184100000141414118410000013F
:1001860041414118410000FF4141413C41003F01CE
:10019600640254000000F894EE27ECBBF1E0FBBFCC
:1001A600EBBFE5BFF8E1F1BDE1BD8DE0A2E0BB2705
:1001B600ED938A95E9F780E098E0A0E6ED93019744
:1001C600E9F7E4E9F1E085919591009761F0A59151
:1001D600B59105901590BF01F00105900D9201971C
:1001E600E1F7FB01F0CFEFE5EDBFE8E0EEBFC0E6DB
:1001F600D2E00C944201AA93BA93EA93FA93EFB72A
:10020600EA93E0916002E2BBA2E6B2E0ED91FD91D5
:100216003196FE93EE93A0916202B0916302A83FDD
:10022600E0E0BE0731F4E0E2E0936002E0E0E09354
:100236006102A0916202B0916302AB3FE0E0BE07AB
:1002460031F4E0E0E0936002E0E2E0936102A09125
:100256006202B0916302A730E1E0BE0731F4E1E04B
:10026600F0E0E0936202F0936302E0916102E2BB88
:10027600E991EFBFF991E991B991A9911895E2E059
:10028600F2E0FBBDEABDE9E0EEBDE0E0EFBDE0E196
:10029600E9BFE0EFE1BBE1E0F0E0E0936202F0935A
:1002A6006302E0E0E0936002E0E2E0936102E0E0F6
:1002B600E0936402E0E8E5BF7894A0916202B09111
:1002C6006302119711F4CC24DD24A0916202B0914F
:1002D6006302AA3AE0E0BE0724F4A734E0E0BE07D2
:1002E6000CF403C0F60138966F018895A09162025E
:1002F600B0916302AA3AE0E0BE0724F4A634E0E037
:10030600BE0714F40C94F00285E08A95F1F7AF93DA
:10031600BF93A4E6B2E0AC0DBD1D4D905D906D900F
:100326007D908D909D90AD90BC90BF91AF91FF93C5
:1003360047FAF2B3F6F90000F2BB46FAF2B3F6F961
:100346000000F2BB45FAF2B3F6F90000F2BB44FA3C
:10035600F2B3F6F90000F2BB43FAF2B3F6F9000085
:10036600F2BB42FAF2B3F6F90000F2BB41FAF2B37D
:10037600F6F90000F2BB40FAF2B3F6F90000F2BB60
:10038600FF91FF9357FAF2B3F6F90000F2BB56FA63
:10039600F2B3F6F90000F2BB55FAF2B3F6F9000033
:1003A600F2BB54FAF2B3F6F90000F2BB53FAF2B319
:1003B600F6F90000F2BB52FAF2B3F6F90000F2BB0E
:1003C60051FAF2B3F6F90000F2BB50FAF2B3F6F9BD
:1003D6000000F2BBFF91FF9367FAF2B3F6F9000053
:1003E600F2BB66FAF2B3F6F90000F2BB65FAF2B3B5
:1003F600F6F90000F2BB64FAF2B3F6F90000F2BBBC
:1004060063FAF2B3F6F90000F2BB62FAF2B3F6F958
:100416000000F2BB61FAF2B3F6F90000F2BB60FA33
:10042600F2B3F6F90000F2BBFF91FF9377FAF2B34D
:10043600F6F90000F2BB76FAF2B3F6F90000F2BB69
:1004460075FAF2B3F6F90000F2BB74FAF2B3F6F9F4
:100456000000F2BB73FAF2B3F6F90000F2BB72FACF
:10046600F2B3F6F90000F2BB71FAF2B3F6F9000046
:10047600F2BB70FAF2B3F6F90000F2BBFF91FF93FC
:1004860087FAF2B3F6F90000F2BB86FAF2B3F6F990
:100496000000F2BB85FAF2B3F6F90000F2BB84FA6B
:1004A600F2B3F6F90000F2BB83FAF2B3F6F90000F4
:1004B600F2BB82FAF2B3F6F90000F2BB81FAF2B3AC
:1004C600F6F90000F2BB80FAF2B3F6F90000F2BBCF
:1004D600FF91FF9397FAF2B3F6F90000F2BB96FA92
:1004E600F2B3F6F90000F2BB95FAF2B3F6F90000A2
:1004F600F2BB94FAF2B3F6F90000F2BB93FAF2B348
:10050600F6F90000F2BB92FAF2B3F6F90000F2BB7C
:1005160091FAF2B3F6F90000F2BB90FAF2B3F6F9EB
:100526000000F2BBFF91FF93A7FAF2B3F6F90000C1
:10053600F2BBA6FAF2B3F6F90000F2BBA5FAF2B3E3
:10054600F6F90000F2BBA4FAF2B3F6F90000F2BB2A
:10055600A3FAF2B3F6F90000F2BBA2FAF2B3F6F987
:100566000000F2BBA1FAF2B3F6F90000F2BBA0FA62
:10057600F2B3F6F90000F2BBFF91FF93B7FAF2B3BC
:10058600F6F90000F2BBB6FAF2B3F6F90000F2BBD8
:10059600B5FAF2B3F6F90000F2BBB4FAF2B3F6F923
:1005A6000000F2BBB3FAF2B3F6F90000F2BBB2FAFE
:1005B600F2B3F6F90000F2BBB1FAF2B3F6F90000B5
:1005C600F2BBB0FAF2B3F6F90000F2BBFF91EF937B
:1005D600E894E2B3E6F9E2BBEF910C946001FFCF39
:00000001FF
